:020000022000DC
:106000000000042009820200498202004B82020043
:106010004D8202004F820200518202000000000007
:106020000000000000000000000000008981020064
:106030005582020000000000A9810200598202007E
:10604000699F02007D6502005B8202005B820200A4
:106050005B8202005B8202005B8202005B820200C4
:106060005B8202005B8202005B8202005B820200B4
:106070005B8202005B8202005B8202005B820200A4
:106080005B820200B17F02005B8202005B82020041
:106090005B8202005B8202005B8202005B82020084
:1060A0005B8202005B8202005B820200D17102000F
:1060B0005B8202005B820200000000000000000022
:1060C0005B8202005B8202005B8202005B82020054
:1060D0005B8202005B8202005B820200AD920200E2
:1060E0005B8202005B8202005B8202000000000013
:1060F000000000005B820200000000005B820200E2
:10610000000000000000000000000000000000008F
:10611000000000000000000000000000000000007F
:10612000000000000000000000000000000000006F
:10613000000000000000000000000000000000005F
:10614000000000000000000000000000000000004F
:10615000000000000000000000000000000000003F
:10616000000000000000000000000000000000002F
:10617000000000000000000000000000000000001F
:10618000000000000000000000000000000000000F
:1061900000000000000000000000000000000000FF
:1061A00000000000000000000000000000000000EF
:1061B00000000000000000000000000000000000DF
:1061C00000000000000000000000000000000000CF
:1061D00000000000000000000000000000000000BF
:1061E00000000000000000000000000000000000AF
:1061F000000000000000000000000000000000009F
:1062000010B5054C237833B9044B13B10448AFF3F0
:1062100000800123237010BDF8360020000000002C
:1062200060D2020008B5034B1BB103490348AFF32A
:10623000008008BD00000000FC36002060D2020093
:10624000154B002B08BF134B9D46A3F5803A002148
:106250008B460F461348144A121A04F06BFC0F4B7E
:10626000002B00D098470E4B002B00D09847002001
:10627000002104000D000D48002802D00C48AFF3A7
:10628000008004F0EDFB2000290001F0FDFF04F088
:10629000D3FB00BF00000800000004200000000045
:1062A00000000000F8360020EC4A0020000000004A
:1062B000000000001F2886BF00F01F00044A4FF0B6
:1062C000A042012303FA00F0C2F80805704700BF9E
:1062D000000300501F2886BF00F01F00044A4FF043
:1062E000A042012303FA00F0C2F80C05704700BF7A
:1062F0000003005070B5554A554E1378554C002593
:10630000356003F0FF01002B00F08280524B1988AA
:10631000524BB3F80900884207D11570B3F8032037
:10632000B3F801306281238101254D4A137883B18E
:10633000494B19884B4BB3F80500884209D100211D
:10634000117049491A681B79226148480B7100F0A5
:10635000FCFE002D5ED1638940F2E24058435FD0DD
:1063600000F06AFF002D47D13B4A404813880133B3
:106370009BB2138000F00EFF3D4908703D48037842
:10638000002B51D03C4B1B6833603C4B1B785BB1FE
:106390003B4A1378052B9BBF137801330023DBB2F4
:1063A0008ABF13701370037032682AB3334B1B78A3
:1063B000002B46D033481378007800283BD043F0B8
:1063C000080331481370326800781378002835D0FC
:1063D00043F0040313702D4B62790978306801256E
:1063E0001D70237943EA0223A27943EA024322681B
:1063F00000F052FD264B1D7026490B78062013BB7A
:10640000FFF768FF0B78B3FA83F35B090B7070BD7D
:106410000D468AE7238940F2E24003FB00009FE734
:10642000284600F009FF9FE71B4B1B78002BBBD0D1
:106430001A4B3360B8E723F00803C2E723F00403E4
:10644000C8E70370C7E7FFF735FFDBE73B3A0020FB
:10645000403A00201A3A0020183A0020303A002032
:10646000173A0020103A00202A3A00206037002016
:10647000503A0020443A0020643A00200A340020B8
:10648000453A0020593A0020583A0020603A00204E
:10649000493A0020003400200B340020053400204D
:1064A00008B5104B1B78E3B90F490B780620ABB940
:1064B000FFF710FF0B78B3FA83F35B090B700B4BFC
:1064C0001A780132D2B2272A88BF25221A70084AC8
:1064D00018781168BDE8084000F05EBCFFF7EAFEDE
:1064E000E8E708BD603A002000340020503A002060
:1064F0004C3A002001F0FEBF70B5074D0024014466
:10650000E0B2834203D90E5D66550134F8E70349D2
:106510000A70034A137070BD683A0020793A00206F
:10652000783A0020F8B5114B1A7802F0FF00E2B17A
:106530000F4A1978DFF840C00E4F1668C9B2002222
:10654000D0B281420AD9B518387812F80C40285CCC
:10655000844202F10102F3D0002006E0002216205E
:1065600001211A7003F0B6F80120F8BD783A002036
:106570005C3A0020793A0020683A0020524BD3F868
:10658000002170B522B10022C3F8002101229A60D7
:10659000D3F80C21002A00F0968000254B4CC3F85C
:1065A0000C51227802F0FF06002A32D0484B2570A9
:1065B0001A7852B31D70474B474C484801221A7055
:1065C000238940F2E24103FB011101F5967100F0CD
:1065D0000DFE434B22681D80424B43481A6062798E
:1065E000237943EA0223A27943EA02433F4A04F1B2
:1065F0001001136000F016FD617D3B4801F01F01A2
:1066000000F0C1FD384800F0C1FDBDE8704000F069
:106610008DBC01259D60D3F80034002B53D0FFF7CB
:1066200081FFC8B1324B4FF4B4502B4398472F4BE6
:106630002C4A304930481B68126809780068257078
:1066400000F02AFC2D4A1378DBB2AB4204D116705D
:106650001F4A137000F0F6FD29490C686378981CF6
:10666000FF2830D8184AD2F80C2422540C6804446D
:10667000150A65700C682044120C82700933214A97
:10668000DBB21370134A107880B11F4B1B786BB1CB
:106690000B681E491B780878C3F38003984212D018
:1066A0000B701B481B49002404700B7013783BB11E
:1066B00000F0DCFD184B002118600D2003F00AF8F3
:1066C000164B01221A7070BD00100040603A002085
:1066D0007A3A00205A3A00201A3A0020F562020065
:1066E000183A00204C3A002060370020543A00202D
:1066F000C0CD0200503A0020643A0020513A0020F8
:106700005C3A0020483A00200A340020583A002021
:10671000443A0020593A00203C3A0020473A0020F1
:1067200008B500F08FFD104B104900221A70104B75
:10673000104A1960104B1A60104B2520187000F099
:106740002BFB0F490F4800F051FD01210D2002F0F5
:10675000C1FF01210C2002F0BDFF01211620BDE880
:10676000084002F0B7BF00BF5A3A0020D6BE898E5B
:106770004C3A002055555500543A0020503A00201C
:1067800090D00300A164020038B51E4C1E4A236855
:106790001D78137805F00F052BB1002313701B4AE9
:1067A0001370FFF7BDFF052D0BD006230222082131
:1067B0002068FFF7A1FE00211620BDE8384002F056
:1067C00089BF00F03FFD2068114B00F10E0200F17F
:1067D00022011C4652F8045B43F8045B8A42F9D15B
:1067E00012881A80082106230222FFF785FE63899A
:1067F0003BB1084B01221A7000F038FD064B1860BF
:10680000D9E738BD643A00205A3A0020443A0020C3
:106810001A3A0020513A00203C3A0020164B1B68DF
:106820001A7802F00302032A03D19A785AB1012A96
:1068300017D0124B1B782BB1114B01221A70114B40
:1068400000221A707047104A53F8031F11605968EC
:106850005160198911819B7A93720C4B01221A7035
:10686000E7E753F8030F0A490860988888809B7906
:106870008B71084BF3E700BF643A00205A3A0020BE
:10688000443A0020453A0020303A00203B3A0020AC
:10689000103A0020173A002010B501210C2002F018
:1068A000F1FE01210D2002F0EDFE0121162002F083
:1068B000E9FE01210C2002F00DFF01210D2002F064
:1068C00009FF0121162002F005FF4FF0A04103242B
:1068D000C1F84C471320FFF7EDFCC1F818470F4CE7
:1068E0000620FFF7E7FC20464FF4E13101F001FEFE
:1068F0000A21204600F0B8FC40F20B1004F0D4F856
:10690000074B0930186040F20B1004F0CDF8054B2E
:106910000930BDE810401860FFF702BFE4410020D5
:106920005C3A0020643A002008B5044800F04EFCB0
:10693000034B002283F8482008BD00BF60370020C9
:10694000143700200A46A72330B400F8053C131280
:1069500000F8033C0D4B00F8042C1C8800F8024C96
:106960001B881B0A00F8013C411F04460023251A1E
:10697000ADB2AA4204D914F8015B2B44DBB2F6E7AE
:1069800083540632024830BC01F099BD183A002009
:10699000E44100200A46BB2330B400F8053C131242
:1069A00000F8033C0D4B00F8042C1C8800F8024C46
:1069B0001B881B0A00F8013C411F04460023251ACE
:1069C000ADB2AA4204D914F8015B2B44DBB2F6E75E
:1069D00083540632024830BC01F071BD183A0020E1
:1069E000E4410020A94B2DE9F74FD3F8002112B163
:1069F0000022C3F80021A64B1B789BB1A54B1A7847
:106A000082B100221A70A44B1868A44B1A1D904240
:106A100002BFA34A12681A6041780931C9B204382A
:106A2000FFF7B8FF9F4B1A7842B100221A709E4BB5
:106A300019789E4B18680438FFF784FF9C4B1A782E
:106A4000984692B100F012FC9A4B1B68C01A9A4B00
:106A5000DA890A235343984207D901210D2002F015
:106A600039FE00210C2002F035FE944C944F25464F
:106A700094F84830D3B3934B1B78BBBB924B1B7835
:106A800003F0FF0693BBDFF85C922288D9F8000080
:106A9000A1690432043804F029F8A06904F00CF864
:106AA00094F8481032460139D3B28B4202F1010208
:106AB0000BDADE1D581C55F826C09E1D45F826C071
:106AC00035F8100025F81300EEE7D9F8003053F838
:106AD000043CBB4207D1FFF757FE95F84830013B15
:106AE00085F84830C4E7FFF799FEF6E7774E784F10
:106AF000DFF8F491304601F0D1FC002800F0F68078
:106B0000304601F0CEFCC0B2A72820D011DC6628A8
:106B100062D0A628EED101220DF105013046FFF723
:106B2000E9FC9DF80530C72BE4D11320FFF7D2FB19
:106B3000E0E7AA2800F0A380CC2800F0A380A928D1
:106B4000D8D1644901223046FFF7D4FCD2E73B7824
:106B500003F0FF0A002BCDD102220DF106013046D1
:106B6000FFF7C8FCBDF806B0BBF5877FC2D20BF1BA
:106B7000050003F099FF0BF101020146044630467F
:106B8000FFF7B8FCBDF806105346524618B28842CB
:106B900003F1010303DA205C0244D2B2F6E7635C3E
:106BA000934214D195F848300C2B08D89A1D25F83B
:106BB000131045F82240013385F848309AE7204603
:106BC00003F07AFFA121304601F070FC92E72046E5
:106BD00003F072FFA821F6E701220DF1050130460E
:106BE000FFF788FC9DF80530BBB33B7803F0FF044A
:106BF000002B7FF47FAF00F025FB334B4FF0010AF1
:106C000087F800A01C702F4B88F800401C70324B96
:106C10001C70324B1C70324B214616201C7002F047
:106C200059FD21460C2002F055FD51460D2002F081
:106C300051FD5146042002F04DFD95F8483004F115
:106C4000010AE4B2A34206D9063455F8240003F041
:106C500033FF5446F1E70023AEE73A78002A3FF4C9
:106C600049AF194A3B701370084AC2F80031C2F8A4
:106C70000C319360134A1370FFF752FD3AE701227B
:106C8000494660E7012202495DE700BF001000406D
:106C90005B3A0020493A0020403A002001340020AD
:106CA0004C3A0020473A0020483A00205C3A002045
:106CB0005A3A00203C3A00201A3A002014370020AB
:106CC000D6BE898E443A0020603A0020E44100207C
:106CD000463A00200B3400203B3A0020173A0020AF
:106CE000513A0020643A00200A3400200E4B1B78F1
:106CF000ABB10E4B1A7892B90D4A0E4810600122C2
:106D00001A700D4C0D4B0E4A1B681268217800F06A
:106D1000C3F82378262B8CBF25230133237040BF73
:106D200020BF03B0BDE8F08F463A0020603A002053
:106D3000643A002005340020503A0020543A0020E4
:106D40004C3A002025280AD026280AD027280AD025
:106D50000A28D4BF023003304000C0B2704702207E
:106D600070471A207047502070470000084BD3F836
:106D7000502562B1074A0221C2F880100022C3F8F0
:106D8000102101221A61D3F81021002AFBD070478C
:106D90000010004000E100E070B506460C46FFF729
:106DA000E5FF4FF080430022C3F8002101221A6062
:106DB000D3F80021002AFBD0324B04220025C3F86F
:106DC0000C25C3F82C55D3F8302542F00102C3F846
:106DD00030250322C3F810253046FFF7B3FF220EFB
:106DE000C3F80805C3F85465C3F824252202C3F884
:106DF0001C254FF48472C3F81425234AC3F81825C0
:106E0000D3F8502642F00102C3F8502640F25B62EC
:106E1000C3F8382540F20312C3F834251B4AC3F8DF
:106E20003C251B4A1168081F106001F8044C1168CA
:106E3000C4F3072048701168C4F3074088701168D4
:106E4000C4F30764CC701168043111600822C3F8E0
:106E50000415C3F804230F4A602182F801130221AC
:106E6000C2F8801111600122C3F800515A60D3F8B2
:106E70000021002AFBD00022C3F80C2101229A60D5
:106E800070BD00BF00100040FB00030255555500C7
:106E90005C3A002000E100E02DE9F041204C0026A2
:106EA000C4F8006215460F469846FFF75FFF1D4A7B
:106EB000C4F804050223C2F8803113600423C4F827
:106EC0000C353846C4F84465FFF73CFF164AC4F851
:106ED00008051168C4F854750323C4F800320B1F69
:106EE000136001F8045C1368C5F307215970136837
:106EF000C5F3074199701368C5F30761D97011682C
:106F00002B0E043111602D02C4F824350123C4F87E
:106F10001C55C4F83C85C4F800612360BDE8F081CD
:106F20000010004000E100E05C3A00200E4B1A68BF
:106F30000E4BC3F804250E4A02210120C2F880102E
:106F4000C3F80002C2F8801111600022C3F81021BA
:106F50001861D3F81021002AFBD00022C3F80021C9
:106F600001225A60704700BF5C3A002000100040C8
:106F700000E100E070B52526002506FB0101E818B8
:106F800090FBF6F406FB14000C5C944204D001352F
:106F9000252DF4D14FF0FF3070BDF8B51F4600230A
:106FA00005460E46FFF7E6FF3A46044603463146DD
:106FB0002846FFF7DFFF031B8442A8BF253318468E
:106FC000F8BD2DE9F04106460D46174698460024C7
:106FD000214643463A463046FFF7DFFF2855013445
:106FE0000C2CF5D1BDE8F081F0B500242346252610
:106FF000C51895F8E151012D1FBFD0F89C7293FB85
:10700000F7F507FB15352D180EBF135595F8BC5134
:10701000155501340B44252C93FBF6F506FB15336F
:10702000E6D1F0BD2DE9FF47002301AEC6E90133EB
:1070300000F2E117044601933846DA1003F0070521
:107040008A5C01332A4102F00102252B00F8012B52
:10705000F3D101F125020023C84311F8015B012D92
:1070600001BFE51800EB010C85F8BCC101338A4271
:10707000F3D1C4F89C32A046052542462946204655
:107080000135FFF7B1FF112D08F12508F5D1B946FB
:107090004FF0000819F8013B012B4DD104F5DE70CB
:1070A000234600250022114613F801C0C44501D132
:1070B000EABB012201312529F6D125339842F1D1CD
:1070C000D5BBC4F8A082BA461AF8013B012B30D1D7
:1070D0002B46D4F8A02231462046FFF772FF00224B
:1070E00013460132B11811F8010C114616F801C00F
:1070F0000131844508BF01230C29F7D10B2AF0D1B7
:10710000BBB9C4F8A45204F5027204F5277142F821
:10711000043B9142FBD10523F21812F8052C823270
:1071200044F822300133112BF6D101200AE0154634
:10713000C3E70135252DC7D108F10108B8F1250FA6
:10714000A8D1002004B0BDE8F08730B50022134676
:10715000DC1003F007050C5D2C41E40742BF8418E6
:10716000013284F8BC310133252BF1D1C0F89C22C7
:107170004B1E00F2E110243113F8012F00F8012B0F
:107180008B42F9D130BDC0F8A81270470023C0F877
:10719000AC327047D0F8AC32D0F8A82225211A447E
:1071A00092FBF1F301FB1323C218C0F8AC3292F842
:1071B000E121012A08D0D0F89C1293FBF1F201FBE7
:1071C0001233184490F8BC311846704770470000DD
:1071D000044B0022C3F84021034B1B6803B118473E
:1071E000704700BF00B001407C3A00200F4B10B543
:1071F00018600F4B0F484FF000640322C0F8804125
:10720000C3F808254FF48032C3F84015C3F80423AF
:1072100004210122C3F80022C3F810156021046084
:1072200080F81B13DA601A6010BD00BF7C3A0020A2
:1072300000B0014000E100E0014BC3F84005704799
:1072400000B00140064B4FF00062C3F88020054BB0
:107250000022C3F840210122DA605A60704700BF63
:1072600000E100E000B001408160704708B500F027
:10727000DBF94FF47A72A0FB0223900A40EA8350B4
:1072800008BD00002DE9F041044600F07DFE314BC1
:10729000314D1A68314E01321A602A68002A4FD1E6
:1072A0002C601B68012B25D12D48DFF8EC802D4F79
:1072B00002F02FFA2C4802F02CFA2C4802F029FA9E
:1072C0002B4802F026FA2B4802F023FA404602F03F
:1072D00020FA384602F01DFA274802F01AFA274829
:1072E00002F017FA264802F014FA264BC3F8008081
:1072F000254B1F60254A136801331360244AE3635A
:107300001168E36A8B4288BF1360154A142000FBA2
:107310000320211D02F00BFA00F040FE33686BB130
:107320002B68DA6AE36A9A4208D21A4B4FF080520D
:107330005A6040BFBFF34F8FBFF36F8FBDE8F0813E
:107340003368002BD6D12B68DA6AE36A9A4298BF79
:107350002C60CFE7F03A0020803A0020503B00201C
:107360008C3A00201C3B0020A03A0020B43A0020B8
:10737000C83A0020DC3A00203C3B0020683B00205B
:10738000543B0020843A0020883A0020003B002033
:10739000043B002000ED00E0083B0020094B0A4AB6
:1073A0001B681268D06A50B9084A1268012A07D8C7
:1073B00033B9074B1868074B1B68C01A7047002089
:1073C000704700BF043B0020803A00208C3A002028
:1073D000343B00207C3B0020064A13681968064BAA
:1073E00019B94FF0FF321A6070471268D268D2683C
:1073F0005268F8E7843A0020343B00202DE9F0473A
:10740000DDE9097496000D4632468046A521206BC1
:10741000994603F08FFB236B043E1E4426F00706BB
:107420006B1E04F13402073513F8011F02F8011B2B
:10743000197809B1AB42F7D1089D042D28BF042566
:107440004FF0000AE562C4E9115A201D84F83BA000
:1074500002F06AF9C5F1050504F1180002F064F9BB
:10746000C4F84CA02461A561646284F850A04A4627
:107470004146304600F050FD206007B13C60BDE859
:10748000F08710B590F8513004463BB9006B02F01C
:1074900091F92046BDE8104002F08CB9012BF9D0DB
:1074A00010BD0000F8B5164B164E1C680546306836
:1074B00004300F4602F05EF96B1C334607D137B13A
:1074C000316811480431BDE8F84002F030B91A685B
:1074D0006419546007D30D4A10681968BDE8F84074
:1074E000043102F030B90A4A10681968043102F018
:1074F0002AF9084B1A68A24288BF1C60F8BD00BF79
:107500007C3B0020803A0020543B0020883A002039
:10751000843A0020343B002030B587B0DDE90B45CC
:107520008DB194B12C63022485F8514005AC0194CF
:107530000A9C02950094FFF761FF2846FFF7A2FE20
:10754000059807B030BD2846FBE72046F9E72DE94E
:10755000F043074685B0900088461646994602F0EB
:107560001AF90546E8B1542002F015F90446A8B10D
:10757000002380F851300D9B056301930C9B029012
:10758000009332464B4641463846FFF737FF2046C8
:10759000FFF778FE012005B0BDE8F083284602F031
:1075A00009F94FF0FF30F6E710B588B0002407AABC
:1075B00006A905A8CDE9054400F052FF059B0293FA
:1075C000069B079A0E490F48CDE900432346FFF773
:1075D000A3FF0D4B186080B100F052FB01280CD1C5
:1075E000402383F31188094B4FF0FF321A60084B98
:1075F0001860084B1C6000F0A1FC08B010BD00BF73
:10760000C6CD020005780200303B0020343B00204C
:10761000503B00207C3B0020024A1368013313607A
:10762000704700BFFC3A0020014B1868704700BF4C
:107630007C3B0020024A136818441060704700BF6A
:107640007C3B00202DE9F84F2E4B1B68002B53D1BB
:107650002D4B1D6801351D605DB92C4A2C4B1168FE
:10766000186810602B4A1960136801331360FFF724
:10767000B3FE294F3B68AB424FF0000607D9274BBA
:107680001B68002B0CBF30460120BDE8F88FDFF8E7
:107690007C90DFF894A0DFF894B0D9F800301B6834
:1076A0001BB94FF0FF333B60E9E7D9F80030DB68E6
:1076B000DC6863689D42F6D304F10408404602F09A
:1076C00059F8A36A1BB104F1180002F053F8E36AF9
:1076D000DAF800201420934200FB03B0414688BF33
:1076E000CAF8003002F023F80D4BE26A1B68DB6A2F
:1076F0009A4228BF0126D0E70A4A13680133136073
:107700000026BCE7FC3A00207C3B0020843A0020A5
:10771000883A0020383B0020343B0020803B00208A
:10772000803A0020F83A0020043B00208C3A0020E8
:107730002DE9F04100F028FC294B1A68013A1A6043
:107740001C682CB1002400F029FC2046BDE8F08123
:10775000244B1B68002BF5D0234D244EDFF8A0806E
:107760001DE0EB68DC68271D04F1180002F002F848
:10777000384601F0FFFFE36A32681420934200FBB1
:107780000380394688BF336001F0D1FF184BE26AAD
:107790001B68DB6A9A4202D3164B01221A602B68DF
:1077A000002BDED10CB1FFF717FE134D2C6844B14E
:1077B000104E0127FFF746FF00B13760013CF9D1B9
:1077C0002C600C4B1B68002BBCD00C4B4FF0805234
:1077D0005A6040BFBFF34F8FBFF36F8F0124B2E7F2
:1077E000FC3A0020F03A00203C3B0020043B002003
:1077F000803A0020803B0020F83A002000ED00E0B5
:107800008C3A0020F8B51B4C1B4F1C4D2368EBB97C
:107810001B4B1B68012B08D91A4B4FF080525A6042
:1078200040BFBFF34F8FBFF36F8F00F011FEFFF724
:10783000B5FD0128E9D9FFF7EFFEFFF7AFFD0128FD
:1078400001D900F00BFCFFF773FFDEE700F09CFBB3
:10785000FB68DE68301D01F08DFF2B68013B2B605B
:107860002368013B236000F099FB3046FFF709FED7
:10787000CCE700BFF43A0020683B0020F03A00203B
:107880008C3A002000ED00E0F8B5194B1A68194B4E
:1078900012B101221A60F8BD174C1A6022682368E1
:1078A00012681B6B9A4204D820682168343100F0BA
:1078B000CDFD124E124B32684FF0140C1F460CFBDC
:1078C00002F158185D5885B1456808316D6845600A
:1078D0000B449D4204BF6B684360142303FB027397
:1078E0005B68DB6823603260D5E7013AE7E700BFF9
:1078F000FC3A0020803B0020803A0020043B00201E
:107900008C3A002010B5064B0C461968183101F06E
:107910001AFF20460121BDE81040FFF7C3BD00BF9C
:10792000803A002038B5084B0D46196814461831C6
:1079300001F0FDFE002C21460CBF28464FF0FF3021
:10794000BDE83840FFF7AEBD803A002038B5C368C7
:10795000DC6804F11805284601F00CFF114B1B6888
:10796000EBB9251D284601F005FF0F4AE36A1168AF
:107970008B4288BF13600D4A1420294600FB032068
:1079800001F0D5FE0A4BE26A1B68DB6A9A4285BFAA
:10799000084B012000201860FFF71EFD38BD294666
:1079A0000548EDE7FC3A0020043B00208C3A00201B
:1079B000803A0020803B00203C3B0020034B1B68AA
:1079C0000360034B1B684360704700BF383B0020D7
:1079D0007C3B002070B50C46054600F0D5FA0F4BF5
:1079E0001A682368591C0FD00D482E680068696812
:1079F000864201D091420ED9521A934209D99B1A5C
:107A000023602846FFF7DAFF002400F0C7FA20467B
:107A100070BD002323600124F7E700BF7C3B0020FA
:107A2000383B0020014B01221A607047803B002048
:107A3000084B186860B9084B1B6853B9074B1868A6
:107A4000074B1B68013B984214BF0120022070477E
:107A5000002070473C3B0020803B0020543B00202E
:107A6000F03A0020054B1B6833B1054B1B68002B17
:107A70000CBF02200020704701207047503B0020BF
:107A8000FC3A0020F8B5044600282BD01B4AC36AF4
:107A90001168C96A8B42164627D28269184D002A9E
:107AA000A1BF3268D26AC2F105028261142202FBD0
:107AB000035342699A4211D1071D384601F05AFE1C
:107AC0003368104ADB6A1168E3628B420BD81420DA
:107AD000394600FB035001F02AFE02E03368DB6AFE
:107AE000C3620120F8BD1360F1E71368406CDC6AE3
:107AF000A0422CBF00200120F4E700BF803A002004
:107B00008C3A0020043B002038B5044608B9002018
:107B100038BD836CC16A426C013B91428364F6D0EC
:107B2000002BF4D1051D284601F024FE636CE362AE
:107B3000C3F10502A261074A11688B4288BF136036
:107B4000054A142000FB0320294601F0F0FD012026
:107B5000DEE700BF043B00208C3A002070B50446ED
:107B600050B3436C994238BF1946C36A8B4223D045
:107B7000826C012A20D18269104DC162002A4FF027
:107B8000140202FB03534269A4BFC1F105018161E4
:107B90009A4211D1061D304601F0ECFD084AE36A15
:107BA000116814208B4200FB03503146BDE8704041
:107BB00088BF136001F0BBBD70BD00BF8C3A0020D0
:107BC000043B0020044B1A681AB119688A6C013210
:107BD0008A641868704700BF803A0020F7B5114CDE
:107BE00000F0D2F92568BDB90F4F104E384601F0AC
:107BF00090FD304601F08DFD0D4B0E4A1F600E4B7F
:107C000010211E60202000950C4B01F0A1FE206089
:107C100010B10B4902F0CEF803B0BDE8F04000F01F
:107C2000BDB900BF083E00208C3D0020A03D0020D3
:107C3000843B00208C3B0020883B0020B83D002086
:107C4000CBCD0200914208B5416000610AD8D21A3A
:107C500083699A420DD2084B011D186801F073FD2B
:107C6000002008BD9A4201D2994202D2011D034B65
:107C7000F3E70120F5E700BF883B0020843B0020AC
:107C800010B588B0FFF7AAFF0E4B18680024B8B1F2
:107C900007AA06A905A8CDE9054400F0EDFB059B60
:107CA0000293069B019302230093079A0649074813
:107CB0002346FFF731FC064B1860001B18BF01205C
:107CC00008B010BD083E0020D0CD0200817D02002A
:107CD0000C3E00207FB50F4C0546206816461A461C
:107CE00080B10529CDE9001602950DDCFFF7BAFE3B
:107CF0000023022808BF089A206818BF1A46694660
:107D000001F05AFE04B070BD0023694601F0E9FE9F
:107D1000F8E700BF083E00202DE9F341164D4FF073
:107D200000082B681A6832B9144A11682960136078
:107D300002B0BDE8F081DB68DC681E68271D3846AC
:107D400001F018FD636A20469847E369012BE8D1EA
:107D5000A36933449E4206D2636024613946286891
:107D600001F0F1FCDDE70023CDF800803246194632
:107D70002046FFF7AFFFD4E7843B0020883B00207C
:107D80002DE9F04F5D4D89B0A9464FF0000A2A68F1
:107D90001368002B4ED0D268D2F800B0584C039331
:107DA000FFF73AFCFFF740FC2268564E039B9042D7
:107DB0008046274640D2FFF7AFFFC4F80080FFF7A8
:107DC000B7FC4FF0010B002204A9306801F0E2FE7D
:107DD0000028DCD0049B002B03DADDE90601059BBB
:107DE0009847049B002BEEDB069C636913B1201DB2
:107DF00001F0C0FCFFF718FC3B689842024603D232
:107E00000390FFF789FF039A049B3A60092BDAD8A5
:107E10000BFA03F313F4047868D113F0C70F4AD1B7
:107E20009B06D0D594F82C30002BCCD1204601F005
:107E3000C1FCC8E79B46B1E720600BB3834538D847
:107E4000FFF776FCD9F80030DB68DC68201D01F014
:107E500091FCE369012B0FD1A1695B46424659446D
:107E60002046FFF7EFFE38B10023CDF800A05A46B8
:107E700019462046FFF72EFF636A20469847A0E781
:107E8000214B1B681A68B2FA82F25209ABEB080167
:107E9000306801F09DFFFFF74BFC002891D11B4B90
:107EA0004FF080525A6040BFBFF34F8FBFF36F8FC8
:107EB00087E70022EAE7A169059B20461944FFF7FE
:107EC000C1FE00283FF47FAF636A20469847E3690C
:107ED000012B7FF478AFA2690599CDF800800A44A0
:107EE000434641462046FFF7F5FE6CE70599A16140
:107EF000134611442046FFF7A5FE64E7843B0020AB
:107F0000B43D0020083E0020883B002000ED00E04A
:107F1000402383F31188FEE74FF0807340E902139A
:107F2000054B40F80C3C6FF0020340F8202C40F861
:107F3000243C4438704700BF117F02000F4C08B545
:107F4000E02384F8223000F06DF80D4B00221A6017
:107F5000D4F888300B4A43F47003C4F8883053686F
:107F600043F040435360236943F01003236100F062
:107F7000F9F8402383F31188FEE700BF00ED00E02D
:107F8000103E002030EF00E0402383F31188024AC6
:107F90001368013313607047103E0020034A1368D2
:107FA000013B13600BB983F311887047103E00202A
:107FB00073B5194B00221A601B680193019BEFF304
:107FC0001186402383F31188144BD3F80445C3F87A
:107FD000002103F580731B680093009BFFF724FBCF
:107FE000241A24F07F44012C04D9FFF73BFD02281A
:107FF00018BF0124002514F1FF3409D225B1084B24
:108000004FF080525A6040BF86F3118802B070BDB5
:10801000FFF718FB0543EEE7401101400010014057
:1080200000ED00E00A4B0B491F22C3F8082501228E
:10803000C3F804230A601A600222C3F84423064BE3
:10804000E02283F811234FF400321A60704700BF1A
:10805000001001400810014000E100E0F0B50546C5
:1080600085B0EFF3108072B6374CA36883B9012353
:10807000A360364B3649D3F880200A402260C3F80B
:108080008010D3F8842062604FF0FF32C3F8842060
:1080900000B962B62F4FD7F80465FFF7C9FC3B461D
:1080A000002841D02C49A94228BF2946721822F045
:1080B0007F420120C7F80803C7F84025274A00205F
:1080C00010601068019001984FF48030C7F80403E5
:1080D000BFF34F8F3DB11D4820BFD0F80071D0F8DD
:1080E00004513D43F8D04FF48030C3F8080300201A
:1080F000106012680392039A194A10601268029283
:10810000029A0122C3F80423D3F804359B1B23F001
:108110007F4088420D4B4FF4003228BF0846C3F819
:10812000802108B1FFF786FAA3685BB1EFF31083F3
:1081300072B6064A21681160616851600022A2602F
:1081400003B962B605B0F0BDC84A002000E100E006
:10815000FC06FFBD00100140FDFFFF004011014083
:10816000001101400748006880F3088862B661B6D4
:10817000BFF34F8FBFF36F8F4FF0E00080F3118894
:1081800000DF00BF00600200064B19680868B0E815
:10819000F04F80F30988BFF36F8F4FF0000080F33A
:1081A00011887047803A0020EFF30980BFF36F8F8A
:1081B000144B1A681EF0100F08BF20ED108A20E93A
:1081C000F04F10604DF8043D4FF0400080F31188EF
:1081D000BFF34F8FBFF36F8FFFF756FB4FF00000D9
:1081E00080F3118808BC19680868B0E8F04F1EF0E9
:1081F000100F08BFB0EC108A80F30988BFF36F8FAF
:10820000704700BF803A00200A490B4A0B4B9B1A6B
:1082100003DD043BC858D050FBDC094809494FF046
:10822000AD32026004300439FBD100F071F8FEF782
:1082300007F800006CD2020000340020F83600205D
:1082400000F8032000080000FEE7FEE7FEE7FEE777
:10825000FEE7FEE7FEE7FEE7FEE7FEE708B5FEF70E
:108260001BFB074C074DFEF7BDFB002000F0D4F9C7
:10827000002CF8D0002DF6D0AFF30080F3E700BF5C
:10828000000000000000000007B501F0C7F901F090
:10829000C2FD104B104C13B1AFF3008020600F4BA8
:1082A0000193012322880E4900930E480023FFF713
:1082B0004EF901F085F9FFF777F9BFF34F8F0A49BF
:1082C0000A4BCA6802F4E0621343CB60BFF34F8FDE
:1082D00000BFFDE7000000000C340020143E002029
:1082E000D8CD02005D82020000ED00E00400FA0536
:1082F000054B1B68082B01BF044B1868B0FA80F0CF
:10830000400918BF002070473001001034010010F0
:1083100008B54FF080430022C3F80C21C3F81021A8
:10832000C3F838254FF0805203F54043D2F80414C7
:10833000C3F82015D2F80814C3F82415D2F80C1489
:10834000C3F82815D2F81014C3F82C15D2F8141459
:10835000C3F83015D2F81814C3F83415D2F81C1429
:10836000C3F84015D2F82014C3F84415D2F82414E9
:10837000C3F84815D2F82814C3F84C15D2F82C14B9
:10838000C3F85015D2F83014C3F85415D2F8341489
:10839000C3F86015D2F83814C3F86415D2F83C1449
:1083A000C3F86815D2F84014C3F86C15D2F8442409
:1083B000C3F87025FFF79CFF10B11B4B1B4A1A60D6
:1083C000FFF796FF18B11A4BFB22C3F81825FFF7E9
:1083D0008FFF48B11749184B0A681B6822F00F023B
:1083E00003F00F0313430B60FFF782FF18B1134B29
:1083F0004FF400721A604FF08043D3F80024D20784
:1084000044BF6FF00102C3F800240D4AD2F888304F
:1084100043F47003C2F88830BFF34F8FBFF36F8F00
:10842000084B094A1A6008BD8C5600404881030079
:1084300000F00040E40E0040580200104096024058
:1084400000ED00E0103400200090D003704770472A
:1084500008B5024B0BB1AFF3008008BD000000006F
:10846000034B0360034B0B6064231360704700BF32
:108470001C3E0020703E0020034B0360034B0B604A
:1084800064231360704700BF004000205440002068
:10849000014B01221A707047183E0020002000F0A6
:1084A00057B808B5002000F05DF808BD002000F0C6
:1084B00093B808B50021084600F078F808BD70B5FB
:1084C0000E46154614467CB1002000F025F858B140
:1084D00022463146002000F091F8241A064403D0C9
:1084E000002000F099F8EEE7281B70BD002000F096
:1084F00093B87047002000F04BB80000044B4FF4D5
:108500007A720021C3E90112024A1A60704700BF63
:10851000E4410020E8CD0200044A4FF4567303FB07
:108520000020007900F00100704700BFF4410020F6
:10853000064A4FF4567303FB002000F108038068DD
:1085400008609A889B798B718A807047F44100207B
:10855000034A4FF4567303FB0020008B704700BFA3
:10856000F441002007B5094A4FF4567303FB00207D
:108570000DF10701103000F00DFA20B19DF8070051
:1085800003B05DF804FBFF20FAE700BFF4410020D0
:1085900010B5054C4FF4567303FB004092B21030F7
:1085A00000F01FFA10BD00BFF441002007B5094AD2
:1085B0004FF4567303FB002089B20DF1070210300F
:1085C00000F02EFA20B19DF8070003B05DF804FB1F
:1085D000FF20FAE7F441002013B502AC064A04F884
:1085E000011D4FF4567303FB002021460122243065
:1085F00000F05FFA02B010BDF441002010B5054C48
:108600004FF4567303FB004092B2243000F051FA4D
:1086100010BD00BFF44100202DE9F041154F4FF48B
:10862000567444433E190020B17800F027FE80467E
:1086300010B10020BDE8F08104F546753D4404F119
:10864000240040222946384400F0CBF9034608B9FB
:108650000120EFE73279D207EBD52A46B1784046C0
:1086600000F0ACFD0028F3D1034B1B68DB07E0D51D
:1086700000BEDFE7F4410020F0ED00E037B5194C13
:108680004FF456720021204602F054FAFF23637122
:108690004FF4E1330125A3600823A3734FF48072E4
:1086A0002B4604F13801009504F1100000F057F951
:1086B00004F50E71284601F0FFF9002320620093B3
:1086C0004FF480722B4604F59C7104F1240000F0F5
:1086D00046F904F52271284601F0EEF9606303B013
:1086E00030BD00BFF441002010B5074C002304F159
:1086F00010002360237100F0F3F904F12400BDE8B9
:10870000104000F0EDB900BFF4410020F7B58B79BF
:10871000022B064615465CD1CB79002B5BD0073B7C
:10872000DBB2F72B57D92F4FBB78002B57D18B7863
:108730003B700C7809230C4413806378242B0DD0F4
:10874000052B1AD12146304600F006FD68B9264BAC
:108750001B68D90700D500BE202027E023782A888F
:1087600013442B8023781C44E7E7A3787B7023789D
:108770002A8813442B8023781C446378042B1AD155
:1087800063790A2B17D123782A8813442B80217808
:10879000164B0093022201332144304600F0A2FB25
:1087A00030B1114B1B68DA0700D500BE03B0F0BD35
:1087B0002B880E332B8040230D4AF978304600F089
:1087C000FDFC50B9084B1B68DB0700D500BE21201B
:1087D000ECE71520EAE71620E8E70020E6E70023AB
:1087E0001B70FFDEF4410020F0ED00E0F6410020B8
:1087F000CC44002038B50C46097801F06003202BEA
:10880000054648D16378A3F12002012A27D8E388DE
:10881000A3B921780023C1F3C0111A4681F00101E8
:10882000284600F07BFC6378202B05D11B4B1BB145
:108830001B490020AFF3008000200FE0072B28BF6A
:108840000723C909164A00F069FC164B4FF0FF31A7
:10885000186801F019FA0028DBD10B2038BD222B53
:1088600015D10023C1F3C0111A4681F0010100F0B7
:1088700055FC0D4B618819710C4B002BDCD0C1F3FA
:108880004002002001F0010101F01AFBD4E70021B1
:1088900000F0D8FCD0E71E20E0E700BF0000000099
:1088A000FC4100200C4A0020F4410020C19E02003F
:1088B0002DE9F0471C4CE2788A42804602D0002025
:1088C000BDE8F0876779DFF870A003F536764FF4DE
:1088D000367504F11009B54216D1144B2BB1238B18
:1088E0009BB213B10020AFF300804023104AE1781F
:1088F000404600F063FC0028E1D10E4B1B68DB070B
:1089000000D500BE2120DBE76119484600F09FF842
:10891000BAF1000F06D0635DBB4203D13946002097
:10892000AFF300800135D6E7F441002000000000DD
:10893000CC440020F0ED00E000000000006920B110
:1089400000231A46194601F037B87047006908B588
:1089500018B14FF0FF3101F097F9012008BD2DE962
:10896000F0410446884617461E46FFF7EFFF0546CE
:1089700068B19DF81830A37300232381C4F80080E8
:108980006381A780E680A3812046FFF7D7FF2846B2
:10899000BDE8F08103899BB270B504460E4613B959
:1089A0000025284670BDFFF7D1FF05460028F7D007
:1089B000E2882368A189304602FB013102F096F873
:1089C000A389A1885A1C92FBF1F301FB13239BB2EC
:1089D000A3812389013B9BB223812046FFF7AEFF91
:1089E000DFE72DE9F0410489A4B205468846164622
:1089F00084B103899A4288BF06894FF0000788BF77
:108A0000B6B2BCB2A64205D941462846FFF7C2FF1E
:108A1000013710B92046BDE8F081EB889844F0E7B3
:108A200038B5034610461A8991420ED29C899D881A
:108A3000DA881B68214491FBF5F405FB141102FB55
:108A4000013102F053F8012038BD0020FCE7038912
:108A500082889A4270B504460E4604D1837B13B9CE
:108A60000025284670BD2046FFF770FF0546002808
:108A7000F6D0E28823686089314602FB003002F0BC
:108A800035F86389A1885A1C92FBF1F301FB13238B
:108A90009BB263812389994215BF2389638901337E
:108AA0009BB216BF9BB2A38123812046FFF746FFEE
:108AB000D7E72DE9F04107460E46144652B19046DD
:108AC00000254545ACB205D031463846FFF7BFFF1B
:108AD000013510B92046BDE8F081FB881E44F0E75F
:108AE00038B50446FFF732FF054630B10023238135
:108AF00020466381A381FFF721FF284638BD00008F
:108B000038B50A4C05462046002300F8013B1022E8
:108B1000FF2102F00FF804F111001022FF2102F0F2
:108B200009F82846BDE83840FFF7DEBD4C45002077
:108B3000C1F1010100231A46C9B200F0EFBA08B52D
:108B400013463AB100231A4600F0CBFF003018BF9D
:108B5000012008BD4FF0FF3200F02EFFF6E70000C5
:108B600083B54FF000089B4CC1469B4D994928683E
:108B7000C4F808904FF0FF32C4E9009901F00AF8F8
:108B80006378062B40F0DE802179257811F07F068E
:108B900040F0AD806279062A43D1E3881A0A022A9E
:108BA00025D0032A28D0012A36D18C4B1B6819689E
:108BB00069B3122366899E4228BF1E46002E2BD021
:108BC000B6F5807FD1D83246854801F08FFF2179F4
:108BD000834A3346C909284600F0A0FA814B4FF07A
:108BE000FF31186801F050F80028BED03BE07B4B05
:108BF0001B6859684B88DDE77B4A9189DBB2994253
:108C00000AD9926852F8231031B10B78D2E7774B2A
:108C10001B68D90700D500BE0021284600F012FBD2
:108C2000A3E7082A05D1724B6D4A1B781370012304
:108C3000D0E7052A04D1A179284600F06DFA94E71F
:108C4000092AE9D1A6792846314600F066FA634A36
:108C5000674B12681E7057689A4657B9634B1B687A
:108C6000DA0700D500BE21792846C909FFF760FF61
:108C70007BE77B8807F109061F44BE4202D3AFF3AE
:108C80000080F0E773780B2B02D133781E44F4E7B1
:108C9000042BE3D17379022BE0D1B37853445A7893
:108CA000FF2ADBD102AA314622F8028D284683F83A
:108CB0000180FFF72BFD0028D0D1BDF806C0BCF124
:108CC000080FCBD933465A78052A08D19978CA09B2
:108CD0000AEBC20201F07F010A4482F811801A787F
:108CE000104480B284451344EDD86644C5E701F0D2
:108CF0001F0101290AD1227A3D4B13445B78002BD6
:108D00008AD13C492846FFF775FD2EE7022E83D114
:108D1000627942B9217A284600F07CFA304A2179FA
:108D20001080334656E7012A04D1217A284600F004
:108D300099FA98E7032A7FF46FAF217A284600F06A
:108D400081FA90E7072B11D12179294BC80901F04D
:108D50007F0203EBC00313445B7C002B7FF405AF61
:108D6000A36862792078FFF7A3FDFEE6012B0CD102
:108D70002078FFF7C5FE0021286800F0B3FD194BED
:108D80000021186800F0AEFDEFE6022B0ED120782E
:108D9000FFF7B6FE0021286800F0A4FD114B00216A
:108DA000186800F09FFDAFF30080DEE6032B3FF470
:108DB000DCAE082B06D16368002B3FF4D6AEA0686A
:108DC0009847D2E6094B1B68DB077FF5CEAE00BEA5
:108DD000CBE600BFDC48002070450020D0340020E6
:108DE0000C4900200C4A0020D4340020F0ED00E0B3
:108DF0004C450020E048002030B5002085B000F050
:108E000089F9184A184D51881346002433F8080B85
:108E10000094526800F09CFD2860F0B10323009399
:108E20002246124B2146012000F092FD104B1860A3
:108E30002B68A3B10F4800F11003C2880293836826
:108E4000019383880093C16800682346FEF764FBA2
:108E5000FFF714FC204605B030BD0E20FBE70F20C5
:108E6000F9E700BF1434002070450020344600208C
:108E70000C4A00206C34002010B54378013B0446B6
:108E80000A46062B1CD8DFE803F00404041B1B046D
:108E90000B00114B0146BDE810401868FFF74FBEAC
:108EA000017999B9836823B10C4B18684AB100F075
:108EB00047FE637923B10A4B1B68DB0700D500BE70
:108EC00010BD1346114600F077FDF2E7024B014654
:108ED0001868FFF734FEECE7704500200C4A0020CC
:108EE000F0ED00E02DE9F843089D07460C4690465A
:108EF000994602266378052B04D1E17801F003013D
:108F0000414508D0104B1B68DA0700D500BE1C2075
:108F100018E00126EEE72146384600F01DF930B989
:108F2000094B1B68DB0700D500BE20200AE0A178B2
:108F3000CB0914BF297089F800102178012E0C4448
:108F4000E7D10020BDE8F883F0ED00E01FB5002375
:108F5000019308238DF80530044BCDE9020101A9E6
:108F60001868FFF7ECFD05B05DF804FB70450020C4
:108F7000024B1B68DB0700D500BE7047F0ED00E038
:108F80000D4B93F8B420014662B10C4A5268C2F30B
:108F900008021AB101220A48FFF7D8BF93F8B4209B
:108FA000002AFBD1012283F8B4200A60BFF36F8F3F
:108FB000BFF34F8F704700BF104A002000ED00E064
:108FC000818F020038B5134D134BEA88AC88297A9B
:108FD000A41AA4B2402C28BF40242A6889B9C3F837
:108FE00000270122C3F80447DA64BFF36F8FBFF391
:108FF0004F8F2B6823442B60EB881C44A4B2EC8079
:1090000038BDC3F800260548C3F80446FFF7B8FF8B
:10901000EFE700BF104A00200070024004700240D9
:1090200038B5104A00F59473451E52F823400E4B94
:10903000182101FB0535142303FB0023E968C3F85D
:109040000017E4B2C3F80447084B03EB8000FFF7B6
:1090500097FFEB682344EB606B8A1C44A4B26C82DC
:1090600038BD00BF00700240104A00202870024046
:10907000114B411E182202FB013110B4CA8B8B8B9D
:109080008C699B1A91F820209BB2934228BF13460B
:109090001422424302F1804202F51C32C2F800461B
:1090A000C2F8043623448B61044B5DF8044B03EB98
:1090B0008000FFF765BF00BF104A00200470024027
:1090C0001FB50023CDE90133039107238DF8080074
:1090D000012101A88DF80530FFF7CEFE05B05DF83F
:1090E00004FB000000221146930003F1804303F5C6
:1090F0001C330132082A59609962F5D1034B0448A8
:109100005962B8229964002101F014BD0070024038
:10911000104A0020012070477047704738B51D463F
:109120000B4C43B1A3800023E38022602172FFF740
:1091300049FF012038BD0748FFF722FF94F8B430FB
:1091400013B9FFF715FFF4E784F8B450F1E700BF57
:10915000104A00205070024010B58878097900F05C
:109160007F035A1E18245443C0090C2202FB0044FA
:10917000104A22441175012202FA03F40E4970B913
:109180000C339A40C1F80423D1F814352343C1F8B5
:109190001435BFF36F8FBFF34F8F012010BD023323
:1091A0009A40C1F80423D1F810352343C1F8103593
:1091B000EFE700BF104A00200070024001F07F007E
:1091C00070B5441E18266643C909104D0C2404FBD3
:1091D00001642C4423820023E260638291B9354408
:1091E0006B7D03F0FF021BB1FFF71AFF012070BD7A
:1091F00000F59470064B43F82020BFF36F8FBFF348
:109200004F8FF3E7FFF734FFF0E700BF104A00206D
:109210000070024091B1CA0901F07F03084A0BBFF8
:1092200003F5887303F5847302EB830352F823007C
:1092300008BF5868003018BF0120704708467047C3
:1092400000700240064B31B901225A65BFF36F8F9F
:10925000BFF34F8F704741F48071C3F81815F5E7DD
:109260000070024031B1044BC3F81815BFF36F8F83
:10927000BFF34F8F704700BF0070024089B101F00B
:109280007F00431E18205843C9090C2303FB01012A
:10929000054B1944488A098A814294BF0020012065
:1092A00070470846704700BF104A00202DE9F04380
:1092B000984B994ED3F80003002385B01C46012536
:1092C0001F4605FA03F101420CD09A199200D2F818
:1092D00000C0BCF1000F05D00C431760BFF36F8FC7
:1092E000BFF34F8F0133192BEBD1E6070BD5FFF7F7
:1092F000F9FE0023012101A8CDE9013303938DF884
:109300000510FFF7B9FD854B23403BB1844B93F823
:10931000B420002A40F0D780FFF72AFE25022CD582
:109320007C4B4FF0000ED3F880C4D3F88474D3F88C
:109330008864D3F88C54D3F89004D3F89414D3F8F9
:109340009824D3F89C34CDF804E08DF80C004FF04D
:10935000060E8DF80D1001A801218DF805E08DF89D
:1093600008C08DF809708DF80A608DF80B508DF8E3
:109370000E208DF80F30FFF77FFD600507D5684B95
:109380001A7A002A40F0A3806648FFF7F9FDE1044D
:1093900007D5634BDA889988914240F2A480FFF7A1
:1093A00011FE5C4F5E4E0D250122AA40A5F10C0373
:1093B0002242D8B227D0142101FB0373A5F10D027C
:1093C000D3F80817182303FB026E03FB0563A3F50C
:1093D00092784FF0000C8EF815C098F80080C9B252
:1093E0008845A3F5947340F08380BEF81210B3F85B
:1093F00000E08E457CD905F58E7347F823C0BFF396
:109400006F8FBFF34F8F0135142DCDD1E2014AD5B7
:10941000404ED6F86C74C6F86C74BFF36F8FBFF310
:109420004F8F0125DFF8F880A94609FA05F33B4282
:10943000E8B216D018216B1E142201FB038302FB35
:109440000562D2F80426B3F81EC0624492B2DA83F1
:1094500001FB0582B3F81EC09288624551D9FFF71F
:1094600007FE0135082DE0D1DFF8B4801125012673
:109470004FF0180906FA05F3A5F110003B42C0B2FF
:109480000ED0A5F1110309FB05F209FB0383A2F538
:10949000C472598A32F808208A4238D9FFF7C0FDD1
:1094A0000135182DE6D1A3020AD50023CDE90133F9
:1094B00003930121032301A88DF80530FFF7DCFC9D
:1094C00005B0BDE8F083002283F8B42026E7DA88EF
:1094D0009988914202D9FFF775FD58E7D988002095
:1094E000FFF7EEFD53E7D9880020FFF7E9FD58E7C5
:1094F000182101FB0262518A1980518AFFF7E0FDB1
:1095000081E7D98B40F08000FFF7DAFDA9E75E75AF
:10951000C6E700BF00700240409C0010FCFB1F002B
:10952000104A00202870024010B50446FEF79AFA4F
:109530000128204603D1BDE8104001F0BDBABDE8C6
:10954000104000F037B9000030B51C4D85B04FF029
:10955000FF3203A9286800F01DFB0028F7D003980C
:10956000037A4468052B05D8DFE803F0030D1014D7
:10957000191FA047039B186808B1FFF7D5FF039890
:10958000FFF7D2FFE3E7C068A047F3E7D0E90301A4
:10959000A047EFE7D0E90412C068A047EAE7D0E9A6
:1095A0000523D0E90301A047E4E7C3690093D0E9AC
:1095B0000523D0E90301A047DCE700BFE84800200D
:1095C0001FB500220421142000F0D8F9074B0849E8
:1095D000186003AB0193022300934FF480620023D1
:1095E0000448FDF7B4FF05B05DF804FBE84800202F
:1095F00028CF020049950200BFF34F8F0549064B63
:10960000CA6802F4E0621343CB60BFF34F8F00BF20
:10961000FDE700BF00ED00E00400FA05124BD3F8AF
:109620004025124B1A604FF080430122C3F81825E1
:109630009A600F4B4FF40031C3F8801003F1C04320
:1096400003F53C534FF48031C3F84813C3F80813B3
:109650005A609A604FF0A0424FF0FF33C2F80835CD
:10966000C2F80838704700BF00A00040EC48002056
:1096700000E100E008B54FF080434E22C3F81C25FE
:10968000FFF7BAFF2F2814D8104B53F820301F2BA8
:1096900086BF03F01F030E4A4FF0A042032908D8EB
:1096A000DFE801F00210080C03F5E073002142F836
:1096B0002310704703F5E0730C21F8E703F5E0731E
:1096C0000421F4E703F5E0730321F0E734CF02004F
:1096D000000300502F2813D80A4B53F820201F2ACC
:1096E00088BF02F01F024FF001038CBF06484FF005
:1096F000A040934011B9C0F80C357047C0F8083548
:10970000704700BF34CF0200000300500021FFF774
:10971000E1BF00F108034FF0FF324360C0E90223CC
:1097200003610023036070470023036170474368AF
:109730004B609A688A609A68516099600368086112
:109740000133036070470A68531C30B50AD10369BE
:109750005A684A6091608B60596003680861013300
:10976000036030BD00F108035C6825689542EFD8BE
:109770002346F9E7D0E9011203698A6082685160E3
:109780005968814208BF5A60002202611A68013A92
:109790001A601868704710B50446FDF73DFF204673
:1097A00001F082F90446FDF7C3FF0CB9FEF74FFE46
:1097B000204610BD10B5044640B1FDF72DFF2046F0
:1097C00001F07AF9BDE81040FDF7B2BF10BD10B549
:1097D0000446FEF7D9FBA46BFEF7E0FBB4FA84F075
:1097E000400910BD70B51546026C866B044642B93F
:1097F00005689DB94068FEF787F965600136A66384
:1098000070BD6DB9806801F071F9A368226C1344D2
:109810006268A360934201D32368A3600020EDE750
:10982000C06801F063F9236CE26821685B421A4466
:109830008A42E2603EBF62689B18E360022DEDD170
:109840000EB1013EEAE73046D8E7034610B41A6C81
:10985000084662B1D9685C681144A142D96024BF4E
:109860001968D960D9685DF8044B01F03FB95DF81B
:10987000044B704770B50446FEF786FB94F84550DC
:1098800004F124066DB2002D14DCFF2384F845306A
:10989000FEF784FBFEF778FB94F8445004F11006C1
:1098A0006DB2002D12DCFF2384F84430BDE8704017
:1098B000FEF774BB636A002BE7D03046FEF746F82C
:1098C00008B1FEF7AFF8013D6DB2DCE72369002B6C
:1098D000E9D03046FEF73AF808B1FEF7A3F8013DAB
:1098E0006DB2DEE738B504460D46FEF74DFBD4E910
:1098F0000F302268A2604343D1181B1A13446160E1
:10990000E3600021FF23A16384F8443084F84530EC
:109910009DB923696BB104F11000FEF717F840B14F
:109920000A4B4FF080525A6040BFBFF34F8FBFF3D6
:109930006F8FFEF733FB012038BD04F11000FFF7F5
:10994000E8FE04F12400FFF7E4FEF2E700ED00E09A
:1099500010B51C4683B10123002908BF2246C4E983
:109960000F0184F84630194622602046FFF7BAFFFF
:109970009DF8083084F84C30204610BDF8B50646F6
:10998000484350300D461746FFF705FF044660B1C7
:10999000002380F8463055B92060C4E90F650121E5
:1099A0002046FFF79FFF84F84C702046F8BD00F179
:1099B00050030360F1E700002DE9FF470026DFF8C0
:1099C000F490019204468A461F46B046FEF7DCFA40
:1099D000A26BE36B9A4201D3022F1AD13A46514649
:1099E0002046FFF7FFFE636A1BB104F12400FDF778
:1099F000ADFF40B12F4B4FF080525A6040BFBFF3D4
:109A00004F8FBFF36F8FFEF7C9FA012004B0BDE896
:109A1000F087019D1DB9FEF7C1FA0020F6E716B9DF
:109A200002A8FDF7CBFFFEF7B9FAFDF7F5FDFEF74B
:109A3000ABFA94F84430FF2B08BF84F8448094F8C4
:109A40004530FF2B08BF84F84580FEF7A7FA01A92F
:109A500002A8FDF7BFFF30BBFEF796FAA26BE36BDF
:109A60009A420ED1FEF79AFA019904F11000FDF71F
:109A700049FF2046FFF7FEFEFDF75AFE48B10126DA
:109A8000A4E7FEF78BFA2046FFF7F4FEFDF750FE41
:109A9000F5E74FF08053C9F8043040BFBFF34F8F54
:109AA000BFF36F8FEBE72046FFF7E4FEFDF740FEC4
:109AB000B3E700BF00ED00E013B5002200900B46B5
:109AC00001201146FFF744FF044638B10023C0E9E6
:109AD0000033C3601A461946FFF76EFF204602B0F6
:109AE00010BDF8B505461746EFF31186402282F304
:109AF0001188806BEA6B904201D3022B1ED195F83E
:109B000045401A4664B22846FFF76CFE631C10D12C
:109B10006B6A0BB9012009E005F12400FDF716FF7F
:109B20000028F7D0002FF5D00120386086F3118887
:109B3000F8BD013464B285F84540EBE70020F5E755
:109B400038B50C46EFF31185402383F31188826BFF
:109B5000C36B93421BD990F8453001325BB28263EC
:109B60005A1C0FD1436A0BB9012008E02430FDF7DD
:109B7000EDFE0028F8D0002CF6D00120206085F3FF
:109B8000118838BD01335BB280F84530ECE7002026
:109B9000F5E700002DE9F04385B00026DFF8E490FA
:109BA0000192044688463746FEF7EEF9A56BDDB113
:109BB00041462046013DFFF748FEA56323696BB18E
:109BC00004F11000FDF7C2FE40B12E4B4FF0805261
:109BD0005A6040BFBFF34F8FBFF36F8FFEF7DEF9C0
:109BE000012005B0BDE8F083019D1DB9FEF7D6F94F
:109BF0000020F6E716B902A8FDF7E0FEFEF7CEF961
:109C0000FDF70AFDFEF7C0F994F84430FF2B08BFBA
:109C100084F8447094F84530FF2B08BF84F84570F1
:109C2000FEF7BCF901A902A8FDF7D4FEF8B9204659
:109C3000FFF7CDFDA8B1019904F12400FDF762FE04
:109C40002046FFF717FEFDF773FD40B94FF0805334
:109C5000C9F8043040BFBFF34F8FBFF36F8F0126A9
:109C6000A2E72046FFF706FEFDF762FDF7E7204674
:109C7000FFF700FEFDF75CFD2046FFF7A8FD00287A
:109C8000EDD0B5E700ED00E02DE9F04385B000250B
:109C9000DFF81C91019104462F462E46FEF774F919
:109CA000A36BEBB1013BA363236813B9FDF78AFFF4
:109CB000606023696BB104F11000FDF747FE40B10D
:109CC0003B4B4FF080525A6040BFBFF34F8FBFF302
:109CD0006F8FFEF763F90125284605B0BDE8F083D4
:109CE000DDF80480B8F1000F03D1FEF757F9002525
:109CF000F2E717B902A8FDF761FEFEF74FF9FDF78D
:109D00008BFCFEF741F994F84430FF2B08BF84F830
:109D1000446094F84530FF2B08BF84F84560FEF797
:109D20003DF901A902A8FDF755FE48BB2046FFF703
:109D30004EFDF8B123683BB9FEF726F96068FDF7E0
:109D4000A1FE0546FEF72AF9019904F12400FDF76A
:109D5000D9FD2046FFF78EFDFDF7EAFC40B94FF034
:109D60008053C9F8043040BFBFF34F8FBFF36F8FEC
:109D7000012793E72046FFF77DFDFDF7D9FCF7E7C4
:109D80002046FFF777FDFDF7D3FC2046FFF71FFDC8
:109D90000028EDD0002D9FD0FEF7F6F8616A19B1CA
:109DA000236B1968C1F105016068FDF7D7FE9CE7D8
:109DB00000ED00E0054B1A6812B19A682AB9012239
:109DC00043F8321003EBC20358607047D44A0020B6
:109DD00070B504460D461646FEF7D6F894F84430A2
:109DE000FF2B04BF002384F8443094F84530FF2B48
:109DF00004BF002384F84530FEF7D0F8A36B2BB9DD
:109E00003246294604F12400FDF78CFD2046BDE8CA
:109E10007040FFF72FBD08B501210320FFF732FC8A
:109E20000320FFF773FC01210420FFF72BFC042023
:109E3000FFF76CFCBDE8084000F000B830B589B011
:109E400008A8002500F81C5D00F054F808A8184B7D
:109E500040F8183D00F076F800F07EF8154B4022EF
:109E600083F827234FF08043D3F83844E20702D524
